:04093100C180C101BF
:10088C007590FF120901A2019290120901A2019226
:10089C0091120901A2019292120901A201929312E2
:1008AC000901A2019294120901A201929512090167
:1008BC00A2019296120901A2019297120901A200BB
:1008CC009297120901A2009296120901A200929528
:1008DC00120901A2009294120901A200929312092A
:1008EC0001A2009292120901A2009291120901A296
:0508FC00009290808EC7
:10090100900000AF82AE83E4FCFD7BE87A80F9F8C9
:09091100D312091B4003A380EA84
:01091A0022BA
:03000000020800F3
:0C080000787FE4F6D8FD758120020847DF
:10091B00EB9FF5F0EA9E42F0E99D42F0EC6480C853
:06092B0064809845F022F3
:10080C0002088CE493A3F8E493A34003F68001F26E
:10081C0008DFF48029E493A3F85407240CC8C333ED
:10082C00C4540F4420C8834004F456800146F6DFBC
:10083C00E4800B0102040810204080900931E47E12
:10084C00019360BCA3FF543F30E509541FFEE493B1
:10085C00A360010ECF54C025E060A840B8E493A378
:10086C00FAE493A3F8E493A3C8C582C8CAC583CAA3
:10087C00F0A3C8C582C8CAC583CADFE9DEE780BE5B
:0109350000C1
:00000001FF
